:1000000000308A00982D0000831A0A28A500030EEC
:10001000A6000F288312A500030EA600A614A50EA5
:100020000408A7002008A8002108A9002208AA00A7
:100030002308AB002408AC0083120B1E21288B1868
:10004000F2288B1E25280B19F82827088400280879
:10005000A0002908A1002A08A2002B08A3002C0850
:10006000A400260E83008312250EA618831609000D
:100070000A108A100A11820711347B34253429347E
:100080004B348934C1343B3401340B34FF34BF3436
:10009000EF34FD340A108A100A1182076334613488
:1000A0006C3420343D34203400340A108A100A1194
:1000B0008207313439342D344A3455344C342D349C
:1000C0003034353400340A108A100A118207233480
:1000D00020344C346F346734203469346E347434D3
:1000E00065347234763461346C343A3420340034FC
:1000F0000A108A100A1182072334203444346134F0
:10010000743461346C346F34673400340A108A10EC
:100110000A1182072334203444346F3477346E3428
:100120006C346F346134643400340A108A100A115C
:1001300082072334203444346934733470346C348B
:100140006134793400340A108A100A11820723348A
:10015000203449346E34763461346C346934643418
:1001600000340A108A100A11820720346D346F346B
:100170006434653400340A108A100A118207283466
:10018000643429346134743461346C346F346734CA
:100190006734653472342C34203400340A108A10E9
:1001A0000A118207643428346F34293477346E346A
:1001B0006C346F34613464342C3420346434283427
:1001C00069342934733470346C34613479340034D4
:1001D0000A108A100A11820763346D3464343A3489
:1001E000203400348B12AE0A8B168B108A1125280E
:1001F0008B12B00B09290B122F08B0002E08B1008A
:1002000031083202031806293108B200AE01B514D4
:100210000B16AD1C2A29B108031D1029BC03122995
:10022000FF30BC00BC08031D2A29FF30BC00831628
:100230000511831205118316851083128510FF3076
:10024000860083160510831205108316051785177F
:10025000630083122D1C6E29B51C3C29B510310892
:10026000CE00B6010A304E02031C3A290A30CE02F3
:10027000B60A32294E08B700003035180130003870
:10028000031D5329351483168510831285143708EE
:10029000CE004E083820A1002108860083160511E3
:1002A000831205116E293510831605118312051569
:1002B000B608031D63290A30CE004E083820A1007D
:1002C000210886006A293608CE004E083820A10091
:1002D0002108860083168510831285108B160B115A
:1002E0008A11252807309F008316050885000330F2
:1002F0008312A000A00B7A291F080C130030F839D4
:10030000031987109D0183169F018312B32D49089D
:1003100083169B009C131C141A088312A10000343E
:1003200083160510831205140830A1000000000098
:100330000000A117AB29A113CD0C03180510031C55
:1003400005142117AB292113A10B9C2900000000E3
:1003500000000510AB290130A0008401840BAE29F8
:10036000A00BAD290E308400840BB429A11B9B295E
:10037000211BA32900344A30840000080319CF2927
:100380000130A100A001A00BC329A10BC2294A3052
:10039000A000A00BC92900000000800BC029003478
:1003A00081010430A000A01DDD29073081018130CA
:1003B00084000008C0390F38800064008130840058
:1003C0000008C039200480008B160B16C0308B0447
:1003D000312E420883169B008312430883169A002D
:1003E0009C131C1583120B138B138B1BF429553094
:1003F00083169D00AA309D009C14C03083128B048C
:100400000A30CA00BB210034CB0164304902031C0E
:100410000D2A6430C902CB0A052ACB08031D132A12
:10042000CA080319192A30304B07CC004C08CD00FC
:100430009021CB010A304902031C222A0A30C9024A
:10044000CB0A1A2ACB08031D282ACA0803192E2A08
:1004500030304B07CC004C08CD009021303049079C
:10046000CC004C08CD009021003483160511831276
:10047000051583168510831285142D10003408305D
:10048000A10000000000851383168513000083126D
:10049000CB0D0513031C4F2A83160517831203186F
:1004A000542A831605138312831685178312851F1A
:1004B000572AA10B412A00008513831685130000DB
:1004C0000517000000000000000085178312851F3B
:1004D000672AA1010000051B211400008513831663
:1004E00085138312051383160513831200340B132F
:1004F0008B138B1B782A83160517000085170000C5
:1005000083120513831605130000831285138316C7
:100510008513A0308312CB003F22483084000008AE
:10052000CA004A08CB003F224708CB003F224908B7
:10053000CB003F2283160513000085178312851F09
:100540009F2A00000000000000008316051700002D
:1005500005308312CA00BB21C0308B0400342D1437
:100560000034AD100330C5004508C9008721C7011C
:100570002108C6004608C700C60101304507C8006B
:100580004808C90087212108C6070318C70A46087A
:10059000A1004708A2002208C3002108C200C5012B
:1005A00045086320C50ACD00902110304502031D87
:1005B000D02A4308C6004208C5000130C7004630B3
:1005C00084000008C8004808C9004708CA0004227F
:1005D0004508C9004708CA0004220D30CD0090210B
:1005E0000A30CD009021AD19F62A352283168517E1
:1005F000051700000000000000008312C501033051
:10060000450203183A2B83160517000085170000D2
:1006100083120513831605130000831285138316B6
:100620008513A0308312CB003F22FF30CB003F2246
:10063000FF30CB003F2202304502031D232B023046
:10064000CB003F22292B02304507C6004608CB00CD
:100650003F2283160513000085178312851F2E2B5A
:100660000000000000000000831605170000831240
:10067000C50AFF2AC101C0018030410203187E2B48
:100680004308C6004208C500C608031D4A2BC5081A
:100690000319562B0230C700FA30CA00BB21C70B22
:1006A0004C2B45080319C603C503442B3108C4006D
:1006B0007F304102031C642B7F304102031D732BEA
:1006C000FF3040020318732B01304007C500003093
:1006D0000318013E4107C6004608C8004508C70088
:1006E000FF30C90077224108C8004008C70044080D
:1006F000C9007722C00A0319C10A3C2BAF2200347B
:100700000408A1000830A000831685158312851DFA
:10071000872BC401A0179C2BA0139C2B0310C40C87
:10072000851DC41720179C2B2013A00B8E2B21088E
:1007300084004408A100B12B013084000030A01BCC
:100740005530A100A10BA22B840B9E2B0D30A01BBA
:100750000330A100A10BAA2BA01B8C2B201B942BD8
:100760008E2B00340B138B138B1BB32BC001400853
:10077000BB20C00ACD0090210E304002031DB72BD4
:10078000C0014008CE20C00ACD00902115304002A3
:10079000031DC12B0D30CD0090210A30CD009021DA
:1007A000C001C008031DEA2B80232108C0000A30C5
:1007B000CA00BB214008CD00902141304002031CFB
:1007C000E82B5B3040020318E82B40082038E92B67
:1007D0004008C0000D30CD0090210A30CD0090219E
:1007E00064304002031D012CC10141087820C10A78
:1007F000CD00902109304102031DF52B0D30AD00D5
:10080000362C6F304002031D122CC1014108862096
:10081000C10ACD0090210A304102031D062C093087
:10082000AD00362C69304002031D232CC101410864
:100830009520C10ACD00902109304102031D172CDB
:100840000B30AD00362CC1014108A320C10ACD00F8
:10085000902109304102031D242C0D30CD00902140
:100860000A30CD0090210130A1004D2CC10141087A
:10087000B120C10ACD00902105304102031D372C63
:100880000D30CD0090210A30CD0090210230C20001
:100890002D08C300E9210030A100A108031DB62BDB
:1008A0000230C000FA30CA00BB21C00B522C0B131F
:1008B0008B138B1B582C00308A0000287A2E0830AE
:1008C000C7002008C800831605170000851783128B
:1008D000851F682C051B0314051F0310A10D0000C4
:1008E0008316851383128513C70B632C8316051794
:1008F00000008312051348080319812C8316051381
:1009000083120000831685178312851F852C000033
:1009100085138316851300008312051383160513B0
:100920008312D12C3522C101C0018030410203184D
:10093000FA2C4108C4004008C3000B138B138B1B17
:100940009E2C8316051700008517000083120513DF
:100950008316051300008312851383168513A030B8
:100960008312CB003F22443084000008C6004608B2
:10097000CB003F224308CB003F228316051700001F
:1009800085170000831205138316051300008312D8
:10099000851383168513A1308312CB003F22A0015B
:1009A0005F2C2108C50083160513000085178312EC
:1009B000851FD82C000000000000000083160517DA
:1009C0000000C03083128B044508A1002108C2003A
:1009D000420A031DEC2CFA2C4208C900CA01042269
:1009E0000D30CD0090210A30CD009021C00A0319AE
:1009F000C10A952CAF227E2EC20110304102031C89
:100A0000052D1030C102C20AFD2C0A304202031823
:100A1000102D30304207C3004308CD009021182D1F
:100A200041304207C3000A30C3024308CD00902181
:100A30000A3041020318232D30304107C300430818
:100A4000CD0090212B2D41304107C3000A30C30255
:100A50004308CD0090210034C00140084A20C00A5C
:100A6000CD00902106304002031D2D2D2F08C1001E
:100A7000FC240D30CD0090210A30CD009021C20120
:100A80002F08C300E921003480232108C300430854
:100A9000CD0090213A3043020318532D30304302E9
:100AA000A100672D672D61304302031C5E2D7B3052
:100AB000430203185E2D4308DF395F2D4308A00071
:100AC00041302002A0000A302007A100672D003429
:100AD00044252108C20044252108C100DD3041021F
:100AE000031D762D4208A1007F2D7F2D4208A00016
:100AF000A00EF030A00520084107A1007F2D003492
:100B000068252108C0004008C90087212108C000CD
:100B10004008C100FC24862E68252108C0006825F5
:100B20002108C1004008C2004108C300E921882E05
:100B300084011F30830507309F0083160510831240
:100B40000510B601B701B801B901BA01BB01FF3008
:100B5000BC00BD01BE01B101B201AE01B401B301DF
:100B60000130660072290230C90087212108AD00DA
:100B7000C90187212108AF002F08B0002330CD0024
:100B800090212030CD0090210530C0000130C100FF
:100B90004008C90087212108C200C208031DD12DC9
:100BA000D62D4208CD009021C00AC82D411CDE2D53
:100BB0000D30CD0090210A30CD0090212330CD00A2
:100BC00090212030CD009021C00140085520C00A5E
:100BD000CD00902109304002031DE52D0D30CD00E0
:100BE00090210A30CD00902119302D02031DFB2DDC
:100BF00003308600122E09302D02031D022E113003
:100C00008600122E0B302D02031D092ED7308600D0
:100C1000122E0D302D02031D102ED5308600122EFF
:100C2000EF30860083168510831285100230C000D5
:100C30009630CA00BB21C00B182E83168510831274
:100C4000851483160511831205110230C0009630F9
:100C5000CA00BB21C00B272E831605118312051570
:100C6000D0292D1D392E0230C2000930C300E921E0
:100C7000B122C0014008E820C00ACD009021053013
:100C80004002031D3A2E80232108BF003F08CD00FB
:100C900090210D30CD0090210A30CD0090214130BF
:100CA0003F02031C5A2E5B303F0203185A2E3F08A6
:100CB00020385B2E3F08A0006D3020020319792EEA
:100CC0006730200203197B2E7030200203197D2E1D
:100CD0002D30200203197F2E2B3020020319822E83
:100CE000723020020319852E773020020319872ED7
:100CF000892EB22B922EB122922E922C922EAF03DD
:100D00002C25922EAF0A2C25922E802D922E8C2DE2
:100D1000922E3F30CD0090210D30CD0090210A3031
:080D2000CD009021392E630083
:02400E00103F61
:084000000F0004000C000A008F
:0442060000003C0078
:0242F200AF001B
:024204000900AF
:02420000CC00F0
:10420A0052006500760020003100650020000000A1
:1042D60034003600340037002E00300034004E0023
:1042E6002F00300039003000340032002E00340038
:0842F600310057005F000000D9
:00000001FF
